:100000000C942A000C9445000C9445000C94450077
:100010000C9445000C9447000C9445000C9445004A
:100020000C9445000C9445000C9445000C9445003C
:100030000C9445000C9445000C9445000C9445002C
:100040000C9445000C9445000C9445000C9445001C
:100050000C94450011241FBECFE5D4E0DEBFCDBF18
:1000600010E0A0E6B0E0ECE3FBE002C005900D92EA
:10007000AA37B107D9F710E0AAE7B0E001C01D9296
:10008000AE37B107E1F70C946B000C9400001F929F
:100090000F920FB60F9211242F933F938F939F933C
:1000A00086B597B520917A0030917B00821B930B27
:1000B00090937D0080937C0086B597B590937B00EC
:1000C00080937A009F918F913F912F910F900FBE57
:1000D0000F901F901895CEE4D4E0DEBFCDBFEE2484
:1000E000FF248FEF87BB88BB0E94970160E0862FBB
:1000F0000E948B0180E88FBD81E08EBDFDBCECBC11
:1001000080E289BF789480E690E00E94F70140E0A9
:100110005AE560E070E029E030E0CA010197F1F7AC
:100120002150304037FFF9CF88B390E8892788BB4A
:1001300080917C0090917D008E159F0541F37C019C
:1001400060E081E00E94D10184EE90E09F938F9364
:1001500080917C0090917D00AA27BB27BC01CD0136
:1001600020E137E240E050E00E945D05DC01CB0178
:10017000BC01CD0120E030E940E050E00E947C0568
:100180003F932F938FE690E09F938F9381E190E0D0
:100190009F938F938E010F5F1F4F1F930F930E94AA
:1001A0001802C8010E94F7018DB79EB70A960FB6D4
:1001B000F8949EBF0FBE8DBFAACF8150F0F708956F
:1001C00081509040E8F708951F938AB38E608ABBF0
:1001D0008AB38F708ABB8BB3846F8BBBDB9882E052
:1001E0000E94DD00D99A81E00E94DD0019B3107FE2
:1001F000D99882E00E94DD00D99A81E00E94DD005A
:1002000089B382958F70182BD998812F99271F91C8
:1002100008951F938AB38E608ABB8AB38F708ABB9E
:100220008BB38C6F8BBB82E00E94DD00D99A81E09A
:100230000E94DD0019B3107FD99882E00E94DD0092
:10024000D99A81E00E94DD0089B382958F70182BC6
:10025000D998812F99271F9108950E94E40088233F
:10026000E4F3089582E00E94DD00D99A81E00E94C3
:10027000DD00D99808950F931F93082F0E942D0138
:100280008AB38E6F8ABB11E08BB381238BBB902F17
:10029000907F8BB3892B8BBB0E9432018BB3812360
:1002A0008BBB802F992724E0880F991F2A95E1F7AF
:1002B0002BB3282B2BBB0E9432011F910F91089565
:1002C0000F931F93082F0E942D018AB38E6F8ABB54
:1002D00011E08BB381238BBB902F907F8BB3892B45
:1002E00088608BBB0E9432018BB381238BBB802F34
:1002F000992734E0880F991F3A95E1F72BB3282B03
:1003000028602BBB0E9432011F910F91089581E05C
:100310000E943B010895882319F08EE090E002C00E
:100320008CE090E0611101960E943B0108951F93BB
:100330008AB38E6F8ABB80E096E30E94E00011E0F2
:100340008BB381238BBB8BB380638BBB0E94320149
:1003500082EC9EE00E94E0000E9432018CE590E079
:100360000E94E0000E9432018CE590E00E94E000D3
:10037000DC980E9432018CE590E00E94E00088E267
:100380000E943B0186E00E943B010E948701612F91
:10039000812F0E948B011F91089582E00E943B01F2
:1003A0000895823050F4603140F48295880F880FB0
:1003B000807C860F80580E943B0108950E942D0189
:1003C0000E94E400992746E0969587954A95E1F7C3
:1003D00099278170907008950E942D010E94E40079
:1003E00099278F73907008950E9460010895CF93AC
:1003F000DF93EC018881882331F089910E94F40118
:1004000088818823D1F7DF91CF910895CF93DF932F
:10041000EC01FC0121968491882339F00E94F401BB
:10042000FE01219684918823C9F7DF91CF91089529
:100430000F931F93CF93DF93CDB7DEB72E970FB6F1
:10044000F894DEBF0FBECDBF0D891E892F89388D70
:10045000698D7A8D86E08C831A83098337FF05C006
:100460008FEF9FE79E838D8304C0215030403E83F1
:100470002D83AE01455E5F4FCE0101960E9454026E
:10048000ED81FE818E179F070CF4FC01E00FF11F38
:1004900010822E960FB6F894DEBF0FBECDBFDF914F
:1004A000CF911F910F9108952F923F924F925F929B
:1004B0006F927F928F929F92AF92BF92CF92DF9274
:1004C000EF92FF920F931F93CF93DF93CDB7DEB7D9
:1004D00062970FB6F894DEBF0FBECDBFEE24FF24A7
:1004E00087011C017E876D872A01CC24DD24FC0155
:1004F000D782C682838181FD68C28FEF9FEF78C269
:100500008D859E8501969E878D87C0FE4BC28F8507
:1005100080538A30D0F49F85903339F4662029F4D3
:10052000C3FC03C0E0E0F1E08DC08AE0689E602C6F
:100530001124FF856F0E20ED620E67FE02C05FE79B
:10054000652EC3FC42C2762C40C2C3FE04C06620A6
:1005500011F441E0642EEF858E2F992787FD909549
:10056000883691058CF5853691050CF06EC0833583
:10057000910509F493C084359105CCF48B32910533
:1005800009F449C08C3291054CF48032910509F48C
:1005900046C08332910509F44AC0FEC18D329105EF
:1005A00009F440C08E32910509F444C0F5C1833688
:1005B000910509F450C0843691050CF08AC0883545
:1005C000910509F4BCC0E8C18037910509F4B1C0B8
:1005D0008137910584F48C36910591F18D36910522
:1005E0002CF48936910509F474C0D6C18F36910573
:1005F00009F49CC0D1C18537910509F4A2C08637A2
:10060000910524F48337910571F1C6C188379105AE
:1006100009F495C0C1C180E190E0C82AD92AE0E27E
:10062000F0E010C080E890E0C82AD92ACEC1E0E40A
:10063000F0E008C088E090E0C82AD92A6624C5C145
:10064000E4E0F0E0CE2ADF2AC0C13FE3E32E7A9453
:10065000F3E6FF873CC1F20182E090E0480E591EAC
:10066000E0807A9434C1F20182E090E0480E591E95
:10067000A081B1817D01C3FE09C0862D992787FD28
:100680009095BC01CD010E9425051FC0FD01019080
:100690000020E9F73197EA1BE88B18C0F20182E0ED
:1006A00090E0480E591E0190F081E02D7F01C3FEBD
:1006B00009C0862D992787FD9095BC01CF010E9426
:1006C0001A0503C0CF010E941105888B9889791AF9
:1006D000FEC0C2FE0AC0F20184E090E0480E591E3E
:1006E00020813181428153810CC0F20182E090E08F
:1006F000480E591E808191819C01442737FD409509
:10070000542F79018A0157FF0CC0E2E0F0E0CE2AB5
:10071000DF2A10950095F094E094E11CF11C011D76
:10072000111D8FEB9FEFC822D92227C098E0988B2C
:1007300008C0E0E4F0E0CE2ADF2AF8E7FF8720E1F6
:10074000288BC2FE0AC0F20184E090E0480E591ED8
:1007500020813181428153810AC0F20182E090E020
:10076000480E591E808191819C01442755277901AB
:100770008A01EFECFFEFCE22DF22CE0101969A8BA9
:10078000898B9889892E9924AA24BB24C801B70192
:10079000A50194010E947C05DC01CB01E989FA895D
:1007A00080838A3024F0FF858F0F815201C0805DE5
:1007B000E989FA898193FA8BE98BC801B701A50110
:1007C00094010E947C0579018A01211531054105BA
:1007D0005105E1F6E98881E090E08C0F9D1FE81A51
:1007E000C60182739070892B09F07A94C6FE0DC001
:1007F000872D992787FD9095E889E03121F42EEF28
:10080000722E780E02C0782E7A94C3FE0FC0262D69
:10081000332727FD30958E2D9927821793072CF0CB
:1008200087EF9FEFC822D92201C06E18C3FE02C015
:10083000761801C07E18C60180789170892B51F41A
:10084000872D7A94181634F4B10180E290E00E946A
:100850003005F6CFC1FE04C0B1018DE290E00BC0BF
:10086000C4FE04C0B1018BE290E005C0C5FE05C026
:10087000B10180E290E00E943005C6FE10C0B101D7
:1008800080E390E00E9430059889903141F4B101F5
:10089000EF858E2F992787FD90950E943005D0FE19
:1008A0000AC0872D7A94181634F4B10180E390E0E1
:1008B0000E943005F6CFC3FE0AC0862D6A94181632
:1008C00034F4B10180E390E00E943005F6CF90E867
:1008D000B92EBC2051F4872D7A94181634F4B10146
:1008E00080E290E00E943005F6CFFF85F33641F4B8
:1008F0008E2DB101992787FD90950E94300540C04B
:100900002F852337B1F488898150888B8F3FC1F1BF
:10091000F70180810894E11CF11CB101992787FD42
:1009200090950E94300598899150988B9F3F81F750
:1009300027C0EF85E33579F4F889F150F88BFF3F54
:10094000F9F0F7018491B10199270E9430050894CC
:10095000E11CF11CF1CF6E010894C11CD11C8989E6
:100960009A898C159D0561F0E989FA898291FA8B43
:10097000E98BB101992787FD90950E943005EFCF53
:10098000BB2069F0872D7A9418164CF4B10180E2EF
:1009900090E00E943005F6CFB1010E943005CC24D2
:1009A000DD2413C09F85953241F481E0C82ED12CFF
:1009B0006624762CEAE0E88B08C0B101FF858F2F12
:1009C000992787FD90950E943005F101838183FF6F
:1009D00004C0ED85FE85F49103C0ED85FE85F081B0
:1009E000FF872F85222309F08BCDF1018681978126
:1009F00062960FB6F894DEBF0FBECDBFDF91CF91E8
:100A00001F910F91FF90EF90DF90CF90BF90AF902C
:100A10009F908F907F906F905F904F903F902F901E
:100A20000895FC0105900020E9F7809590958E0FC0
:100A30009F1F0895FC010590615070400110D8F788
:100A4000809590958E0F9F1F0895FC016150704016
:100A500001900110D8F7809590958E0F9F1F0895F3
:100A60000F931F93CF93DF938C01EB018B81992719
:100A700081FF1CC082FF0DC02E813F818C819D8132
:100A80002817390764F4E881F9810193F983E88331
:100A900006C0E885F985802F0995892B39F48E8168
:100AA0009F8101969F838E83C80102C08FEF9FEFC5
:100AB000DF91CF911F910F910895629FD001739F95
:100AC000F001829FE00DF11D649FE00DF11D929FEA
:100AD000F00D839FF00D749FF00D659FF00D992729
:100AE000729FB00DE11DF91F639FB00DE11DF91F4D
:100AF000BD01CF0111240895A1E21A2EAA1BBB1B30
:100B0000FD010DC0AA1FBB1FEE1FFF1FA217B307D9
:100B1000E407F50720F0A21BB30BE40BF50B661FEF
:100B2000771F881F991F1A9469F7609570958095B3
:0C0B300090959B01AC01BD01CF01089520
:100B3C00446520706572696F646574696A640069E4
:0A0B4C007320253575202563730022
:00000001FF
